:03000000020B0CE4
:0300030002800375
:03000B0002800B65
:08001300308A0302801301454D
:03001B0002801B45
:0300230002802335
:03002B0002802B25
:10003000A18CA184C187C1E9C1F6A1E2C108A19444
:10004000C1C70202E9C0D0C0E0C2D3C2D4B184D1DA
:10005000C7B40D020193B42002212EB43F04313302
:10006000014DB45111C082C083901458D1F6D08391
:10007000D082C2AA212EB448043152014DB452029A
:10008000219BB453024131B441024167014D743D9B
:10009000B18C22E8C0E0D1E07453B18C7450B18CC3
:1000A000118EA881C0F0D18718D1E0120AEC118E10
:1000B000E6D18718D1E0120AF2118EE6A2E7E43306
:1000C000D191D1E0120AFD118EE583D187E582D16D
:1000D00087E43143A88118E6D18774013143E9D11F
:1000E0008774023143EAD18774033143EBD18774BB
:1000F000043143ECD18774053143EDD18774063167
:1001000043EED18774073143EFD187B1A5D1E074B5
:1001100050B18C120AF2118EC3E5819404F8C082AA
:10012000C083120BA9D083D082D0F0D0E0F8D0E009
:10013000D0D032C082C083B1A5901CD9D1F6D08373
:10014000D08222C0E0D1E07452B18CD0E0D19111C4
:100150008E22C000C001C0F0C082C083901423D1A1
:10016000F6D083D082E4D187743AB18CD1E0E8D163
:1001700087D1E0E9D1877802790E2185E8D18774AB
:100180003AB18C7910D1E0E6D18708D9F8B1A5B899
:1001900080EAB1A5D0F0D001D00022C0F0D1E07447
:1001A00042B18C118EE5F0D187D1E07450B18C74DE
:1001B00053B18C7457B18C118EE8C0E0A881181827
:1001C00018E6D187D1E0C082C083901011A8A85151
:1001D00027901014A8B85127901017A8895127907C
:1001E000101CA8885127901021A8985127901026FC
:1001F000A88751277454B18C7430B18C118EE58C62
:10020000D187E58AD187D1E07454B18C7431B18C37
:10021000118EE58DD187E58BD187B1A5D083D082B2
:10022000D0E0F8D0F0014DD1F6118EE8D187D1E0C1
:1002300022C0F0E8C0E0E581C39404F8C082C08326
:10024000901401D1F6120BA9E581C39406F8A68398
:1002500018A682901412D1F608120BA9D083D0826E
:10026000D0E0F8D0F0014DE8C0E0C0F0A881181847
:10027000C082C083901448D1F6B1E2400EF6B1A519
:10028000D083D082D0F0D0E0F8014D9008AFD1F605
:10029000D083D082D0F0D0E0F8014DC082C08390EE
:1002A0001290D1F6B184B41B0A9012D9D1F6D08342
:1002B000D08222B43AEEB1E240EFF8B1E240EAF582
:1002C00083B1E240E4F582B1E240DEB4010A90126B
:1002D000F4D1F6D083D082220841E1B1E240CAF0E5
:1002E000A3D8F8B1E240C241A44387807589117553
:1002F000985043885274007064E57BA97AAA79AB60
:10030000786301556302CC63031DB50108B502058E
:10031000B503028048C28E758D00758B0020B0FD3C
:1003200020B0F220B0EF20B0EC20B0E930B0FDD228
:100330008E20B0FD30B0FD20B0FD30B0FDC28EE5A6
:100340008B33E58D33F404F5F0F57B6455F57AE5F0
:10035000F064CCF579E5F0641DF578E5F0F58D7580
:100360008921D28E22C082C08390153CD1F6901490
:100370008DE4936029A3D1E0B18C7804D1E0D8FC5E
:10038000E493F5F0A3E493A3A3A3C082C083F58212
:1003900085F083E4D1F6B1A5D083D08280D49015C6
:1003A00067D1F6D083D08222C082C083900816D154
:1003B000F6B184D1C7B41B0A9008AFD1F6D083D070
:1003C0008222B43F239016B9D1F6900843D1F6B1FA
:1003D00084B41B05D083D08222901B93D1F6901C4D
:1003E000D9D1F6D083D08222B45307901338D1F6F6
:1003F000813790130DD1F6900853D1F6D083D08277
:10040000D1E9C082C0839007ECD1F6D083D082D1ED
:100410000850069008AFD1F622740DB18CC082C08E
:100420008390131AD1F6D083D0827400C0E0740098
:10043000C0E0C082C08322900853D1F6D083D0821E
:10044000C082C083D1E99007ECD1F6D083D082D1AD
:1004500008C082C083500C9008AFD1F6B1A5D083FC
:10046000D08222C28A30B30A901350D1F6D083D002
:100470008222900870D1F6B184D1C7B41B0A9008CB
:10048000AFD1F6D083D08222B44C0575B80080037A
:1004900075B8049013C6D1F6D083D08275813874B4
:1004A00000C0E07400C0E0E4C3780079017A007B0A
:1004B000007C007D007E007F00C28AD2B375A884D4
:1004C000737A10B1A57820D1E9743AB18C7420B157
:1004D0008CE493F6D1877420B18CA308B830F2B1C4
:1004E0008C7820E6547FF5F0C39420500375F020FB
:1004F000E5F0B18C08B830EBB1A5B1944002DAC593
:10050000B1A522C083C082B1A59007F8D1F6D082F0
:10051000D083C083C082D108B1A54007B1A5D0E087
:10052000D0E0229008AFD1F6D082D083B1A522C00E
:1005300082C08390123BD1F6D083D082D1E9743A45
:10054000B18CD1E07428B18CE0D187C082C0839097
:1005500008A0D1F6B1E220D50C400AD083D082F0B9
:10056000B1A5A3A13C901262D1F6D083D082227AA9
:1005700012B1A5EAC0E0F11FD0E0FAB1944002DA6E
:10058000F2B1A5223098FDC298E599223099FDF587
:1005900099C29922C0E0C3309808E599B41B03D3EF
:1005A000C298D0E022C0E0740DB18CD0E022B184BA
:1005B000D1C7C3C2D5C2D2B40D03D2D522B41B0257
:1005C000B322B40803D2D222B47F0280F8C0F0F57F
:1005D000F0D1A94009C5F0B18CC5F0D0F022D0F01F
:1005E00080CCB1AE30D50122500122C4F5F0B1AEBD
:1005F00020D20F30D506C2D5E5F0C42250012245E5
:10060000F0227408B18C80DAC0E0E8C0E0E9C0E014
:10061000EAC0E0EBC0E0B1AEF8405D20D55A20D290
:10062000F5B1AEF9405220D52B30D2067408B18C0A
:1006300080E4B1AEFA404120D52130D2067408B131
:100640008C80DEB1AEFB403020D51A30D220740849
:10065000B18C80DE7583008882801D758300E8C4BC
:1006600049F58280138883E9C44AF582800AE8C488
:1006700049F583EAC44BF582D0E0FBD0E0FAD0E044
:10068000F9D0E0F8D0E022C0E0C4D191D0E0D1911F
:1006900022540F240383B18C223031323334353667
:1006A000373839414243444546C3C0F09430F5F0F1
:1006B000940A4006E5F09407F5F0E5F0C354F060C5
:1006C00001D3E5F0D0F022C0F0F5F0C39461400B07
:1006D000941A5007C3E5F09420F5F0E5F0D0F0222D
:1006E000C0E07420B18CD0E022C0E0E583D187E582
:1006F00082D187D0E022C0E0E4932098156010A258
:10070000E7547F3099FDF599C2994003A380E9D061
:10071000E022C298E599B41BDF740DB18C80F0D152
:10072000E9E493A3FBC083C08290102B93FAEB9073
:10073000113B93FE54FC0303FFEE5403D082D0839D
:10074000FE14600FC0E0E493A3FCD0E0146004E466
:1007500093A3FDF185C082C083900F02F1ADEFF845
:10076000D0E0D0F0C0F0C0E0FEE5F0FFE814C33305
:1007700075F07EC0F075F007C0F09008C373D083A9
:10078000D082B1A522743AB18CD1E0EBD187D1E00F
:10079000BE0104790B8011ECD187D1E0BE0204794F
:1007A000088005EDD1877906D1E0D9FC227808EAE6
:1007B000930A18A2E7547FB18C400280F2D1E0D8AE
:1007C000FC223E4C6F633D003A20285665727369E7
:1007D0006F6E20312E302920436F6D6D616E643E47
:1007E000004C6F636174696F6E2028003D4465663C
:1007F00061756C74293A20004E6577206D656D6FC8
:10080000727920706F696E746572206C6F636174A9
:10081000696F6E3A20000D533D53696E676C652019
:10082000537465702C204E3D4E6F726D616C2028A4
:1008300064656661756C74292C203F3D48656C7059
:10084000203E00507265737320616E79206B65796C
:100850003A20000D0D52756E2066726F6D206D6529
:100860006D6F7279206C6F616374696F6E20280000
:100870000D0D496E74657272757074207072696FB7
:10088000726974793E204C3D4C6F772C20483D486E
:10089000696768202864656661756C74293A200070
:1008A0002920204E65772056616C75653A2000201E
:1008B00020436F6D6D616E642041626F7274656478
:1008C000210D0021A921BB21C021C521CA21D5218B
:1008D000DC21E221E921F54100410C4110411441A4
:1008E00017411A411D41204123412B4132413641DC
:1008F00039413C41404143419D414F4156415D4159
:100900006141684177417E4185418C4190419741E9
:10091000A641B441C741CE41D6745212058CEB5466
:100920000712069122744012058C745212058CEB4A
:10093000540112069122EC20E705EC120687229062
:100940000FBEE493A360F3F8C39C70041206F62272
:10095000E493A330E7FA80EAEC547823C4F8EC542B
:1009600080601590112BE893900F973582F5825097
:100970000205831206F68006E82420120687742EEC
:1009800012058CEC540712069122EC20E708C33FB5
:10099000FF500D0E800AF404FCEFC39CFF50011EB3
:1009A000EE120687EF12068722EE54F8F8EBC40326
:1009B000540748120687EC1206872251F831192293
:1009C00051F831362251F831252251EC51DD51E6F2
:1009D000EC12068722313651DD51EC223136EDFC26
:1009E00021CC51F251DD31582251F251DD742F12D8
:1009F000058C31582251F8313651DDEDFC318A2217
:100A000051EC51DD51E6EC12068721F93119410212
:100A10003125410251EC2251F22231582231362245
:100A200031252251EC744212058C22311951DD31ED
:100A30008A22313621F931192251FD22315821F90A
:100A4000318A2251D751EC742B12058C51FD223181
:100A50001951DD51EC22311951DD31362231192184
:100A6000CC313651DD311922ECC0E0EDFC3136518C
:100A7000DDD0E0FC313622313651DD312522312501
:100A800051DD51EC22312551DD313622312521CC89
:100A9000315851DD51F22251FD51DD51E6EC120683
:100AA00087ED1206872251F851D751EC742B1205AD
:100AB0008C51FD2251F851D751EC742B12058C74D6
:100AC0005012058C51F22251F851D751FD2251D7C5
:100AD00051FD51DD51EC22744012058C22742C1210
:100AE000058C1206E022742312058C227441120533
:100AF0008C22744312058C2251EC51DD22C083C03C
:100B0000829014881206F6D082D08322758130C27A
:100B1000D3C2D41202E9D299C29878081205A5D896
:100B2000FE900BDC1206F6908000C082C083900716
:100B3000C21206F6D083D0821206E9C082C083902A
:100B400007C81206F61205841206C7F52090148D08
:100B5000E493604BB52040A3E493C0E0A3E493D0BA
:100B6000F0C082C083F58285F0831206F61205A5D7
:100B7000D083D082A3E493F522E4A393F521D0237C
:100B8000D024900B2AC082C083852482852383C011
:100B900021C02222020B2AA3A3A3A3A3020B50D09D
:100BA00083D0821205A5020B2AE9C0E0EAC0E0EB7F
:100BB000C0E0ECC0E0EDC0E0EEC0E0EFC0E0868356
:100BC00018868212071FD0E0FFD0E0FED0E0FDD0F3
:100BD000E0FCD0E0FBD0E0FAD0E0F9220D202020AC
:100BE0000D20202020202020200C57656C636F6D85
:100BF0006520746F20746865206E657720616E646F
:100C000020706F737369626C79206576656E2069F8
:100C10006D70726F7665642038303331206D6F6E81
:100C200069746F722F64656275676765720D6279AA
:100C3000205061756C2053746F6666726567656ECF
:100C4000206F6E2031342D4F43542D393120666F83
:100C500072206E6F20676F6F6420726561736F6EB4
:100C60002077686174736F657665722E2E2E0D0D78
:100C700054686573652061726520736F6D65206FC0
:100C80006620746865206665617475726573206F8F
:100C90006666657265642062792074686973207085
:100CA0006172746963756C617220646562756767EF
:100CB00065723A0D0D2020202020446F776E6C6FF6
:100CC00061642070726F6772616D732066726F6D00
:100CD00020504320202020202020202020557365F4
:100CE000722D467269656E646C696E65737321213D
:100CF0002121210D202020202052756E2050726F5E
:100D00006772616D202020202020202020202020BC
:100D100020202020202020202020202055736573B3
:100D2000206E6F2065787465726E616C2052414D43
:100D30000D20202020202020284E6F726D616C2C09
:100D4000206F722073696E676C652D7374657029EE
:100D50002020202020202020203C4553433E206B93
:100D6000657920697320737570706F727465640D96
:100D700020202020204C69737420617373656D629C
:100D80006C6520636F64652066726F6D206D656DA4
:100D90006F727920202020206175746F6D617469F5
:100DA0006320626175642072617465206465746596
:100DB0006374696F6E0D20202020204865782044E0
:100DC000756D7020616E6420456469742065787467
:100DD00065726E616C2052414D20202020204F6EA4
:100DE0002D6C696E652068656C702028747970655B
:100DF00020273F27290D0D486F77657665722C20D7
:100E0000796F7520646F6E27742067657420736F27
:100E10006D657468696E2720666F72206E6F7468E6
:100E2000696E272E2E2E202054686520636F64651E
:100E300020666F72207468697320646562756767E5
:100E400065720D726571756972657320717569746B
:100E500065206120626974206D6F726520726F6F0A
:100E60006D207468616E20697320747970696361A4
:100E70006C20666F722061206465627567676572B9
:100E80002C206275742069742077696C6C20616C09
:100E90006C0D66697420696E746F2061203237367C
:100EA000342028384B2078203829204550524F4D87
:100EB0002E0D0D4E4F20436F707972696768742153
:100EC000212020506C6561736520646973747269B8
:100ED0006275746520667265656C792E20204D619F
:100EE0006B65206173206D616E7920636F70696539
:100EF0007320617320796F752077616E742E0D0DEC
:100F00000D004143414CCC4144C420414444C341C1
:100F10004A4DD0414ECC434A4EC5434CD24350CCAF
:100F200044C14445C34449D6444A4EDA494EC34AB3
:100F3000C24A42C34AC34A4DD04A4EC24A4EC34A2D
:100F40004EDA4ADA4C43414CCC4C4A4DD04D4FD648
:100F50004D4F56C34D4F56D84D55CC4E4FD04F5296
:100F6000CC504FD0505553C85245D4524554C95215
:100F7000CC524CC352D25252C3534554C2534A4D21
:100F8000D0535542C2535741D05843C8584348C420
:100F90005852CC3F3FBF0050B054434FCE50B15396
:100FA000434FCE50B249C550B349D043B0543243F9
:100FB0004FCE5053D744B84143C3FDC2FE00E04179
:100FC00043C38153D0824450CC834450C88050B036
:100FD0009050B1A050B2B050B399534255C6CD54C1
:100FE00048B2C85432434FCECC544CB2CB5243419A
:100FF0005032C8CA5243415032CC8C5448B08A5403
:101000004CB08D5448B18B544CB1F0C2D05053D732
:10101000A849C5B849D089544D4FC48854434FCED0
:101020009853434FCE8750434FCE005A0E48732BF0
:101030002B2B2B2B2B2B2B2B2B2B2B3000437521CE
:1010400021212121212121212121212E0E676E061E
:10105000060606060606060606060638006A700A32
:101060000A0A0A0A0A0A0A0A0A0A0A330E5D5D5DBA
:101070005D5D5D5D5D5D5D5D5D5D5D3B0012121200
:101080001212121212121212121212410E8F8F8F9E
:101090008F8F8F8F8F8F8F8F8F8F8F3E005D354C0F
:1010A0004C4C4C4C4C4C4C4C4C4C4C7C0E124F24ED
:1010B0004C4C4C4C4C4C4C4C4C4C4C4C004C4F8085
:1010C00080808080808080808080805D0E4C2B5767
:1010D000924C4C4C4C4C4C4C4C4C4C12001C1C1527
:1010E0001515151515151515151515630E191984F2
:1010F0008888888888888888888888600078781FA9
:10110000278B8B2727272727272727530E5353194A
:101110004C4C4C4C4C4C4C4C4C4C4C530053531C76
:101120004C4C4C4C4C4C4C4C4C4C4C000206080C5F
:101130000E101214161B1E20232425AD066F3939FC
:10114000464949595959595959595963066F3939B5
:1011500046494959595959595959596306AD39168A
:101160000E111109090909090909096306AD3916A2
:101170000E1111090909090909090966061A1F163C
:101180000E1111090909090909090966061A1F162C
:101190000E1111090909090909090966061A1F161C
:1011A0000E111109090909090909096606226916BA
:1011B0001F92867A7A7A7A7A7A7A7A660622A14DAC
:1011C0008386867E7E7E7E7E7E7E7E9B06969D16B6
:1011D0000E111109090909090909092606225D4D9F
:1011E000AD8E8E76767676767676762606423D2FAC
:1011F0002B373733333333333333334606423D39BA
:101200000E111109090909090909094606423D3962
:101210005711115252525252525252A506111139BF
:101220000E11110909090909090909A9068989394C
:101230001A898971717171717171710D4564697467
:10124000696E672045787465726E616C2052414DFD
:101250002E2E2E3C4553433E20746F2071756974C9
:101260000D00202045646974696E672066696E69A7
:10127000736865642C2074686973206C6F63617493
:10128000696F6E20756E6368616E6765640D0D0031
:101290000D0D426567696E20617363696920747220
:1012A000616E736D697373696F6E206F6620496E2E
:1012B00074656C2048455820666F726D61742066B5
:1012C000696C652C206F72203C4553433E20746F3F
:1012D0002061626F72740D0D00446F776E6C6F61E8
:1012E000642061626F727465642062792075736531
:1012F000720D0D000D0D0D0D446F776E6C6F6164F6
:1013000020636F6D706C657465640D0D0052756EB1
:10131000206E6F726D616C6C79000D4E6F7720726C
:10132000756E6E696E67207468652070726F677283
:10133000616D2E2E2E0D0D0052756E20696E20737C
:10134000696E676C652073746570206D6F646500ED
:101350000D0D5468652073696E676C652073746544
:10136000702072756E20666561747572652077698C
:101370006C6C206E6F742066756E6374696F6E207E
:10138000756E6C65737320494E5431202870696EF8
:1013900020233133292069730D636F6E6E6563748A
:1013A000656420746F2067726F756E64206F7220A1
:1013B0006F74686572776973652068656C64206C0A
:1013C0006F772E0D0D000D4E6F772072756E6E6962
:1013D0006E6720696E2073696E676C652073746533
:1013E00070206D6F64653A20203C5245543E3D6448
:1013F000656661756C742C203F3D48656C700D0D01
:1014000000536B697070696E67202D2D2D2D2D2D69
:101410003E004E6578742077696C6C206265202DE3
:101420002D3E000D4C6F633A2020496E7465726E3C
:10143000616C2052616D204D656D6F727920436F34
:101440006E74656E74730D004E6577204163632082
:1014500056616C75653A20000D5175697420736989
:101460006E676C652073746570206D6F64652C20E9
:101470006E6F772072756E6E696E67206E6F726D1B
:10148000616C6C792E0D0D0044505452003F1506CE
:1014900003655214B103A844150F029B4E14BE05F8
:1014A000034814D304C14C14F2056F451529052FC8
:1014B000002052756E2070726F6772616D00204E51
:1014C0006577206D656D6F7279206C6F63617469EB
:1014D0006F6E00204845582044756D70204D656D35
:1014E0006F727920746F207468652053637265652C
:1014F0006E00204C69737420617373656D626C7942
:1015000020636F6465002048656C703F3F3F00209A
:10151000446F776E6C6F61642070726F6772616D7B
:101520002066726F6D205043002045646974206509
:10153000787465726E616C2072616D000C54686520
:10154000736520636F6D6D616E64732061726520D9
:1015500063757272656E746C7920737570706F72DA
:101560007465643A0D0D000D416C6C206E756D65EF
:10157000726963616C2076616C7565732061726558
:101580002073686F776E20696E206865782E202042
:101590005072657373696E67203C4553433E206B00
:1015A00065792077696C6C2065786974207468654A
:1015B0000D63757272656E7420636F6D6D616E641C
:1015C0002C206576656E207768696C65206C697380
:1015D00074696E672F64756D70696E672E20204D7B
:1015E0006F73742070726F6D707473207265717593
:1015F00069726520610D73696E676C65206368614F
:101600007261637465722C207479706963616C6CAB
:101610007920746865206669727374206C657474CF
:101620006572206F662074686520646573697265F1
:1016300064206F7074696F6E2E0D0D466F72206995
:101640006E666F726D6174696F6E2072656761722C
:1016500064696E67207468652073696E676C652DB8
:10166000737465702072756E20666561747572653D
:101670002C0D7479706520273F27207768656E20D0
:1016800061736B6564202753696E676C652D737495
:1016900065702F4E6F726D616C27206265666F7288
:1016A000652072756E6E696E672074686520707251
:1016B0006F6772616D2E0D0D000C546865207369A3
:1016C0006E676C6520737465702072756E20666538
:1016D000617475726520616C6C6F777320796F75BA
:1016E00020746F206578656375746520796F7572F5
:1016F0002070726F6772616D2066726F6D206D650C
:101700006D6F72790D6F6E6520696E73747275639B
:1017100074696F6E20617420612074696D652C207E
:101720007768696C65206D6F6E69746F72696E673A
:1017300020746865207265676973746572732061CF
:101740006E6420696E737472756374696F6E732E44
:101750000D4974206974204E4F5420612073696DC7
:10176000756C6174696F6E2C207468652070726F7F
:101770006772616D2069732065786563757465644F
:101780002062792074686520383033312F3531205C
:1017900070726F636573736F722E0D457874657226
:1017A0006E616C20496E746572727570742023319D
:1017B000206D7573742062652068656C64206C6FA1
:1017C0007720746F206D616B652074686520736984
:1017D0006E676C6520737465702066756E637469DE
:1017E0006F6E2E0D0D44657370697465206174749D
:1017F000656D70747320746F206D616B6520746803
:10180000652073696E676C652073746570207275EE
:101810006E20636F6D70617469626C6520776974A6
:101820006820616C6C2070726F6772616D732C0D33
:1018300074686572652077696C6C20616C7761797A
:101840007320626520736F6D652062617369632028
:101850006C696D69746174696F6E7320647565205D
:10186000746F20697473206E61747572653A0D0D22
:1018700020312D2045787465726E616C20496E743C
:10188000657272757074202331206D757374206ECB
:101890006F742062652064697361626C65642C20DA
:1018A000652E672E204D4F562049452C2338316830
:1018B0000D20322D2054696D6572202331206D7505
:1018C000737420626520636F72726563746C792033
:1018D00067656E65726174696E6720207468652043
:1018E00062617564207261746520666F722074682D
:1018F000652073657269616C20706F72740D20339E
:101900002D20544920616E642052492077696C6C07
:10191000206E6F7420776F726B206E6F726D616CCA
:101920006C792C20652E672E20323030333A204AD5
:101930004E422052492C323030332C2075736520B2
:10194000736B69702E2E2E0D20342D20496E746518
:101950007272757074732077696C6C206E6F74206E
:101960006765742073657276696365206F7220778E
:10197000696C6C20696E746572727570742074681D
:10198000652073696E676C6520737465700D203512
:101990002D2041626F757420333020627974657335
:1019A000206F66207370616365206D7573742062AB
:1019B00065206C65667420617661696C61626C6536
:1019C000206F6E2074686520737461636B210D2035
:1019D000362D203F3F3F20204F7468657220707283
:1019E0006F626C656D73206D617920616C736F201F
:1019F00065786973742C2028746869732070726F1D
:101A00006772616D20697320465245452C20796FBD
:101A100075206B6E6F77290D0D506572686170735C
:101A20002074686520776F727374206C696D6974B7
:101A30006174696F6E206F66207468652073696ECB
:101A4000676C6520737465702072756E20697320F1
:101A5000746861742069742074616B657320610D12
:101A600076657279206C6F6E672074696D6520747D
:101A70006F2065786563757465206576656E207383
:101A8000686F727420706965636573206F66206388
:101A90006F64652E20204974206973207265636F1E
:101AA0006D6D656E64656420746861740D61206E8F
:101AB0006F726D616C2072756E2062652061747446
:101AC000656D7074656420666972737420746F202C
:101AD000657374696D6174652077686572652074DB
:101AE00068652070726F6772616D20676F65732023
:101AF0006173747261792C0D74686520617474650A
:101B00006D707420612073696E676C6520737465F5
:101B1000702061742074686520626567696E6E6903
:101B20006E67206F662074686520717565737469CF
:101B30006F6E61626C6520636F64652C20776974D9
:101B40006820610D68617264636F7079206F662030
:101B500074686520617373656D626C79206C69735C
:101B600074696E672066696C65206F6E2D68616EA2
:101B70006420666F72206D656D6F7279206C6F6383
:101B80006174696F6E207265666572656E63652E3D
:101B90000D0D000C4265747765656E207374657079
:101BA000732C20746865206D6F6E69746F72207578
:101BB000736573206162736F6C7574656C79204E08
:101BC0004F20696E7465726E616C206F722065784B
:101BD0007465726E616C206D656D6F72792E0D4843
:101BE0006F77657665722C2061626F757420333073
:101BF000206279746573206F6620737461636B2053
:101C00007370616365206D757374206265206C6507
:101C1000667420617661696C61626C652E2E2E0D92
:101C20000D447572696E6720612073696E676C651B
:101C300020737465702072756E2C207072657373DA
:101C4000696E672052455455524E20726570656129
:101C50007465646C792077696C6C206265207468A7
:101C60006520757375616C20636F757273650D6F98
:101C70006620616374696F6E2E2020486F776576E9
:101C800065722C206F74686572206F7074696F6E56
:101C9000732061726520617661696C61626C652E8A
:101CA0000D0D2020202020202020202020205479CD
:101CB00070696E6720273F272077696C6C20646904
:101CC00073706C617920746869732068656C70202A
:101CD00073637265656E0D0D0053696E676C6520E8
:101CE0005374657020436F6D6D616E64733A0D0DB2
:101CF000203C5245543E202020205072696E7420B2
:101D000053746174757320616E64206578656375C2
:101D1000746520746865206E65787420696E7374CC
:101D200072756374696F6E0D203C53504143453E9C
:101D3000202045786563757465206E657874206928
:101D40006E737472756374696F6E20772F6F75741C
:101D500020737461747573206C696E65730D202037
:101D6000273F272020202020446973706C61792050
:101D700074686973206F6E2D6C696E652068656C80
:101D8000700D202027522720202020205072696EBD
:101D900074206F7574205370656369616C2046759B
:101DA0006E6374696F6E20526567697374657273D0
:101DB0000D202027482720202020204865782064F7
:101DC000756D7020696E7465726E616C2072616DE4
:101DD0000D20202753272020202020536B697020BE
:101DE0007468697320696E737472756374696F6E59
:101DF0000D202027412720202020204368616E6786
:101E0000652074686520416363756D756C61746FDE
:101E10007227732076616C75650D2020275127206D
:101E200020202020517569742053696E676C6520ED
:101E3000537465702C20636F6E74696E75652065D0
:101E40007865637574696E67206E6F726D616C6C16
:041E5000790D0D00FB
:00000001FF
